:10000000E3288030A100FE30962001309620753024
:10001000A6003030AE28A101A117AE00FE30962018
:100020002E089628A01124080319A0150530A30056
:100030002730A800103028200330A800E8302820FE
:10004000A80164302820A8010A30282029082F2878
:10005000A7002A08A6002908A500C2202508A50097
:10006000A3030319A0112408031939282302031834
:1000700040282508031DA011A0194028303E9628CD
:100080000800A30024080319DE2823089620A403EF
:100090004228AC00061186118316061186110F3016
:1000A000860583122C08A01873283E30A6008030E5
:1000B000AE203330AB0087201330A6008830AE204E
:1000C00087206430AD2087206430AD202230AB0023
:1000D0008720283072200C30722006307220A01445
:1000E0002C0873282014AB00201C81288611033CA7
:1000F000031C862886200730A600D030AE200314CB
:1001000008002014FE3C031994288615201C20109A
:1001100006150F3086052B08F03986040611AB0E44
:10012000201887283230AD202C08DE28A11B492852
:10013000080083178001840AFF3E031D9A28DE28E9
:10014000A801A700FF30A707031CA807031CDE288F
:100150000330A600DF30AE20A228A601E83EA500AD
:10016000A609FC30031CB728A5070318B428A50767
:100170000000A60FB4282518BD28A51CC128000022
:10018000C1280800AA01A9011030AB00260DA90D55
:10019000AA0D2708A9022808031C280FAA02031881
:1001A000D8282708A90728080318280FAA0703102A
:1001B000A50DA60DAB0BC6282508DE2883138312D8
:1001C000031300000800A00183168113203084006F
:1001D000603083129A20A030840050309A20203062
:1001E000840030309920F33083168500FF3086007C
:1001F00020308400603083129A20A0308400503078
:100200009A2020308400303099200130A800F4304A
:10021000A12001206C304920613049206430492000
:10022000653049206E3049203A3049208030A100A5
:10023000C0300B201030A4005F304120C830A02017
:10024000AF0A0319B00A8030A100C0300B202F087C
:10025000A400FF3041202F08103A3004031D1E294E
:100260008030A10080300B200E30A40020304120CF
:100270008030A10080300B2050304920723049205E
:10028000653049207330492049202030492073309F
:10029000492074304920613049207230492074303F
:1002A000492053290929061C5629532901204B307E
:1002B00049206F3049206D3049207430492020306A
:1002C00049206930492065304920213049200511F5
:1002D0008511B001AF010F30A800A030A120861811
:1002E000962985158030A10080300B204E304920A2
:1002F0006930492065304920743049202030492038
:1003000076304920613049206C30492073304920D3
:10031000492070304920653049206C3049206530D3
:1003200049206E30492021304920022A0515073026
:100330003002D03003192F020318A7298618A129EB
:10034000A7290130A020AF0A0319B00A9729073066
:100350003002D03003192F020318ED298030A1009C
:1003600080300B20733049206E30492065304920A1
:100370006C30492068304920653049206930492077
:10038000643049203D30492020304920A401300804
:10039000AA002F08A90012206D30492053304920AF
:1003A000B008031DEC2964302F020318EC298030BB
:1003B000A100C0300B206830492065304920492019
:1003C0006C30492020304920733049206E3049205C
:1003D000653049206C304920022A0511851580308E
:1003E000A10080300B205430492065304920203056
:1003F00049206C304920613049204920743049201F
:0C04000021304920532953296300042AAD
:02400E00503F21
:00000001FF
